:020000040000FA
:100000001DEF1BF012001200E9EF00F012000100DA
:100010008C36000000010000A2000000400EE66ED9
:10002000E66A740EE66E70EC1AF0E552E552E5529F
:100030009F8AD08E9D9AF29CF29E1200D9CFE6FF45
:10004000E1CFD9FF020EE126DE6ADD6AFD0EDBCFCD
:10005000F6FFFE0EDBCFF7FF0800F55015E0FD0EB2
:10006000DBCFF6FFFE0EDBCFF7FF0800F550E66EA4
:1000700055D8E552DF2A010E01E3DB2AFD0EDB2A0B
:10008000FE0E01E3DB2AE2D7DECF14F0DDCF15F060
:1000900014C0F3FF15C0F4FF020EE15C03E200D0D0
:1000A000E16AE552E16EE552E7CFD9FF1200D9CF00
:1000B000E6FFE1CFD9FF020EE126DE6ADD6AFD0E22
:1000C000DBCFE9FFFE0EDBCFEAFFEF5014E0FD0EC1
:1000D000DBCFE9FFFE0EDBCFEAFFEF50E66E1ED866
:1000E000E552DF2A010E01E3DB2AFD0EDB2AFE0EBC
:1000F00001E3DB2AE4D7DECF14F0DDCF15F014C026
:10010000F3FF15C0F4FF020EE15C03E200D0E16AE8
:10011000E552E16EE552E7CFD9FF1200D9CFE6FFF5
:10012000E1CFD9FFACA2FED7FE0EDBCFE6FFE4ECB9
:100130001AF0E552E552E7CFD9FF12000D0EE66E38
:10014000EDDFE5520A0EE66EE9DFE5521200D9CF87
:10015000E6FFE1CFD9FFE65207010451021902E19F
:100160000551031901E1F8D702C7E9FF03C7EAFF08
:10017000022B000E0323EFCFDFFF980E025D010E6E
:10018000035904E3700E026F010E036FDF5000D0BD
:10019000E552E552E7CFD9FF120007017E51EA6A26
:1001A000000FE96E060EEA22EF50836E780EE96EBC
:1001B000070EEA6E7C51EE247C6F7D51EE207D6F40
:1001C0007E51EE207E6F7F51EE207F6F1151E5E072
:1001D0001200DACFE4FFE2CFDAFFE9CFE4FFEACFA3
:1001E000E4FFF6CFE4FFF7CFE4FFF5CFE4FFF3CF72
:1001F000E4FFF4CFE4FFFACFE4FF00EE00F0140ECA
:10020000E80403E3EECFE4FFFBD700EE14F0140E96
:10021000E80403E3EECFE4FFFBD7E6529EAA2DD01D
:10022000A9EC1AF00701116FABA407D0AB9E818136
:100230000F2B000E1023AB8E01D08191ABA207D003
:10024000AB988183AB880D2B000E0E2301D08193D8
:10025000ACA2FED7070104C7E9FF05C7EAFF042BDC
:10026000000E052311C7EFFF980E045D010E05591E
:1002700004E3700E046F010E056FE55200EE27F0E7
:10028000140EE80403E3E5CFEDFFFBD700EE13F017
:10029000140EE80403E3E5CFEDFFFBD7E5CFFAFF4B
:1002A000E5CFF4FFE5CFF3FFE5CFF5FFE5CFF7FFAF
:1002B000E5CFF6FFE5CFEAFFE5CFE9FFE5CFDAFFCF
:1002C0001100D9CFE6FFE1CFD9FFFF0EE76EFD0E9B
:1002D000DBCF14F0FE0EDBCF15F0E7501416156AD5
:1002E0001450A96EFD0EDBCF14F0FE0EDBCF15F01F
:1002F00015C014F0156A030E1414AA6EA69EA69CCF
:10030000A680E80EE66E030EE66EE66AE66A48EC44
:1003100007F0E552E552E552E552A85000D0E5520B
:10032000E7CFD9FF1200D9CFE6FFE1CFD9FF020E08
:10033000E126FD0EDBCF14F0FE0EDBCF15F015C06D
:1003400014F0156A030E1414AA6EFF0EE76EFD0E6C
:10035000DBCF14F0FE0EDBCF15F0E7501416156A54
:100360001450A96EFC0EDB50A86EA69EA684A69C17
:10037000F2AE04D0F29E010EDE6EDD6A550EA76E5F
:10038000AA0EA76EA682A1A8FED7A198A694D9CF3F
:10039000E9FFDACFEAFF010EEE1801E1ED5001E1CD
:1003A000F28E020EE15C02E2E16AE552E16EE55294
:1003B000E7CFD9FF1200D9CFE6FFE1CFD9FFFB0E7F
:1003C000DBCFE9FFFC0EDBCFEAFFEF5022E0FB0EB4
:1003D000DBCFE9FFDB2AFC0EDBCFEAFF01E3DB2A00
:1003E000EF50E66ED950FD0FE96EFF0EDA20EA6E8F
:1003F000EECF14F0EDCF15F0020EEE26000EEF2238
:1004000014C0E6FF15C0E6FF8EDFE552E552E55267
:10041000D6D7E552E7CFD9FF1200D9CFE6FFE1CF1B
:10042000D9FF020EE126D950FD0FE96EFF0EDA204A
:10043000EA6EFF0ED880EE54030EED5401E223D095
:10044000FD0EDBCFE6FFFE0EDBCFE6FF3ADFE55227
:10045000E552DE6EDD6AD9CFE9FFDACFEAFFEE5072
:10046000ED1001E110D0DFCFE6FF58DEE552FD0EC2
:10047000DB2AFE0E01E3DB2AD9CFE9FFDACFEAFF60
:10048000EE50ED10D0E1E80EE66E030EE66EE66A81
:10049000E66A48EC07F0E552E552E552E552020EF5
:1004A000E15C02E2E16AE552E16EE552E7CFD9FF95
:1004B0001200D9CFE6FFE1CFD9FF040EE1260701F4
:1004C000600E006F010E016F00C7E6FF01C7E6FF77
:1004D000FD0EDBCFE6FFFE0EDBCFE6FF94EC15F062
:1004E000E552E552E552E55200C7E6FF01C7E6FFD7
:1004F00062EC1AF0E552E552F3CFDEFFF4CFDDFFF8
:10050000D9CFE9FFDACFEAFF020EEECFDBFF030E11
:10051000EDCFDBFF020EDBCF14F0030EDBCF15F0C7
:10052000040E145C000E15580AE2300EE66EF6DD7D
:10053000E552020EDB2A030E01E3DB2AEBD700C7EC
:10054000E6FF01C7E6FFB3DDE552E552F3CFDEFF7C
:10055000F4CFDDFF040EE15C02E2E16AE552E16EF8
:10056000E552E7CFD9FF1200D9CFE6FFE1CFD9FF9F
:100570000E0EE126F90EDBCFDEFFDBCFDDFFF80E3E
:10058000DB50000802E3070E08D0F80EDB50160817
:1005900002E2170E02D0F80EDB28E66ED950080FE3
:1005A000E96EDACFEAFFE552E750EE6EED6A020E31
:1005B000DB6A030EDB6AFB0EDBCF14F0FC0EDBCF35
:1005C00015F0FD0EDBCF16F0FE0EDBCF17F00A6A3A
:1005D0000B6A0C6A0D6A14C005F015C006F016C04F
:1005E00007F017C008F060EC11F0010A33E1F90ED2
:1005F000DBCFE9FFDB2AFA0EDBCFEAFF01E3DB2AE0
:100600002D0EEF6EFB0EDBCF14F0FC0EDBCF15F0E2
:10061000FD0EDBCF16F0FE0EDBCF17F00A6A0B6A79
:10062000800E0C6EBF0E0D6E14C005F015C006F0E6
:1006300016C007F017C008F05DEC10F0FB0E05C007
:10064000DBFFFC0E06C0DBFFFD0E07C0DBFFFE0E6E
:1006500008C0DBFFFB0EDBCF14F0FC0EDBCF15F088
:10066000FD0EDBCF16F0FE0EDBCF17F00A6A0B6A29
:100670000C6A0D6A14C005F015C006F016C007F02C
:1006800017C008F057EC11F0010A4AE1FB0EDBCF6E
:1006900014F0FC0EDBCF15F0FD0EDBCF16F0FE0ED6
:1006A000DBCF17F00A6A0B6A800E0C6E3F0E0D6EE0
:1006B00014C005F015C006F016C007F017C008F00A
:1006C00060EC11F0010A2CE1146A156A200E166E16
:1006D000410E176ED950FB0FE96EFF0EDA20EA6E5D
:1006E000EECF05F0EECF06F0EECF07F0EFCF08F03B
:1006F00014C00AF015C00BF016C00CF017C00DF0B6
:100700005DEC10F008C0EDFF07C0EDFF06C0EDFF87
:1007100005C0EFFF020EDB06030E01E2DB06B6D7D3
:10072000FB0EDBCF14F0FC0EDBCF15F0FD0EDBCFA4
:1007300016F0FE0EDBCF17F00A6A0B6A200E0C6E65
:10074000410E0D6E14C005F015C006F016C007F07E
:1007500017C008F060EC11F0010A2EE0FB0EDBCFB1
:1007600014F0FC0EDBCF15F0FD0EDBCF16F0FE0E05
:10077000DBCF17F00A6A0B6A200E0C6E410E0D6E6D
:1007800014C005F015C006F016C007F017C008F039
:100790000AEC10F0FB0E05C0DBFFFC0E06C0DBFF11
:1007A000FD0E07C0DBFFFE0E08C0DBFF020EDB2ADA
:1007B000030E01E3DB2AB4D7020EDBCF14F0030EE5
:1007C000DBCF15F0D950080FE96EDACFEAFF1450ED
:1007D000EE261550ED22010EF36E040EF3CFDBFF73
:1007E000050EDB6A040EDBCF06F0050EDBCF07F04B
:1007F00045EC0FF00A0E05C0DBFF0B0E06C0DBFF59
:100800000C0E07C0DBFF0D0E08C0DBFF040EDBCFB4
:1008100014F0050EDBCF15F0080EDBCF16F0090E35
:10082000DBCF17F015501718E8AE02D0173404D0FC
:100830001650145C175015582EE20A0EDBCF14F038
:100840000B0EDBCF15F00C0EDBCF16F00D0EDBCF51
:1008500017F00A6A0B6A200E0C6E410E0D6E14C062
:1008600005F015C006F016C007F017C008F00AEC36
:1008700010F00A0E05C0DBFF0B0E06C0DBFF0C0EEE
:1008800007C0DBFF0D0E08C0DBFF040EDB2A050EE0
:1008900001E3DB2ABBD70A0EDBCF18F00B0EDBCF50
:1008A00019F00C0EDBCF1AF00D0EDBCF1BF00A6A2D
:1008B0000B6A0C6A400E0D6E18C005F019C006F0E8
:1008C0001AC007F01BC008F00AEC10F005C014F0C5
:1008D00006C015F007C016F008C017F0D950FB0F7E
:1008E000E96EFF0EDA20EA6EEECF05F0EECF06F0ED
:1008F000EECF07F0EFCF08F014C00AF015C00BF0F0
:1009000016C00CF017C00DF074EC0FF008C0EDFF2E
:1009100007C0EDFF06C0EDFF05C0EFFFFB0EDBCF0C
:1009200014F0FC0EDBCF15F0FD0EDBCF16F0FE0E43
:10093000DBCF17F00A6A0B6A200E0C6E410E0D6EAB
:1009400014C005F015C006F016C007F017C008F077
:1009500060EC11F0010A13E0FB0EDB6AFC0EDB6AAF
:10096000800EF36EFD0EF3CFDBFF3F0EF36EFE0E37
:10097000F3CFDBFF020EDB2A030E01E3DB2A020EBC
:10098000DBCF14F0030EDBCF15F00001800E151441
:100990005FE0F90EDBCFE9FFDB2AFA0EDBCFEAFFDF
:1009A00001E3DB2A300EEF6EF90EDBCFE9FFDB2A25
:1009B000FA0EDBCFEAFF01E3DB2A2E0EEF6E080E04
:1009C000DBCF14F0090EDBCF15F0800E151414E008
:1009D000020EDBCF16F0030EDBCF17F0080EDB5054
:1009E000165C146E090EDB501758156E020E14C0FB
:1009F000DBFF030E15C0DBFF040EDB68050EDB68B2
:100A0000040EDBCF14F0050EDBCF15F0020EDBCFAA
:100A100016F0030EDBCF17F017501518E8AE02D012
:100A2000153404D01450165C1550175811E2F90E05
:100A3000DBCFE9FFDB2AFA0EDBCFEAFF01E3DB2A9B
:100A4000300EEF6E040EDB06050E01E2DB06D8D792
:100A5000040EDB6A050EDB6A040EDBCF14F0050E14
:100A6000DBCF15F0080EDBCF16F0090EDBCF17F049
:100A700015501718E8AE02D0173404D01650145C85
:100A80001750155801E3ACD0FB0EDBCF05F0FC0E80
:100A9000DBCF06F0FD0EDBCF07F0FE0EDBCF08F05C
:100AA000F1EC10F0060E06C0DBFF070E07C0DBFFFF
:100AB000300EE76E060EDBCF14F0070EDBCF15F01D
:100AC000E7501426000E1522F90EDBCFE9FFDB2AD2
:100AD000FA0EDBCFEAFF01E3DB2A14C0EFFF040EBE
:100AE000DBCF14F0050EDBCF15F0020EDB5014182F
:100AF00003E1030EDB5015180BE1F90EDBCFE9FF24
:100B0000DB2AFA0EDBCFEAFF01E3DB2A2E0EEF6EC3
:100B1000060EDBCF06F0070EDBCF07F045EC0FF03B
:100B20000A0E05C0DBFF0B0E06C0DBFF0C0E07C074
:100B3000DBFF0D0E08C0DBFF05C014F006C015F08A
:100B400007C016F008C017F0D950FB0FE96EFF0E72
:100B5000DA20EA6EEECF05F0EECF06F0EECF07F02A
:100B6000EFCF08F014C00AF015C00BF016C00CF05F
:100B700017C00DF073EC0FF008C0EDFF07C0EDFFDC
:100B800006C0EDFF05C0EFFF146A156A200E166E51
:100B9000410E176ED950FB0FE96EFF0EDA20EA6E98
:100BA000EECF05F0EECF06F0EECF07F0EFCF08F076
:100BB00014C00AF015C00BF016C00CF017C00DF0F1
:100BC0005DEC10F008C0EDFF07C0EDFF06C0EDFFC3
:100BD00005C0EFFF040EDB2A050E01E3DB2A3CD73C
:100BE000F90EDBCFE9FFFA0EDBCFEAFFEF6A0E0E5C
:100BF000E15C02E2E16AE552E16EE552E7CFD9FF3E
:100C00001200D9CFE6FFE1CFD9FF060EE12607019A
:100C1000809DFB0EDBCF05F0FC0EDBCF06F0FD0E5A
:100C2000DBCF07F0FE0EDBCF08F020EC11F004C0A4
:100C3000DEFF05C0DEFF06C0DEFF07C0DDFFDD52C0
:100C4000DD52F90EDBCF06F0FA0EDBCF07F045ECF4
:100C50000FF005C014F006C015F007C016F008C06C
:100C600017F0FB0EDBCF1CF0FC0EDBCF1DF0FD0EF2
:100C7000DBCF1EF0FE0EDBCF1FF0D9CFE9FFDACFBE
:100C8000EAFFEECF24F0EECF25F0EECF26F0EFCF47
:100C900027F024C004F025C005F026C006F027C0C8
:100CA00007F05AEC0FF005C020F006C021F007C095
:100CB00022F008C023F020C00AF021C00BF022C0AF
:100CC0000CF023C00DF01CC005F01DC006F01EC0C6
:100CD00007F01FC008F073EC0FF005C018F006C055
:100CE00019F007C01AF008C01BF018C00AF019C0AC
:100CF0000BF01AC00CF01BC00DF014C005F015C0AD
:100D000006F016C007F017C008F05DEC10F0F1EC2B
:100D100010F0040E06C0DBFF050E07C0DBFF1E0E41
:100D2000E66E010EE66ED9CFE9FFDACFEAFFEECF2D
:100D3000E6FFEECFE6FFEECFE6FFEFCFE6FF2EECCD
:100D400016F0146E060EE15E14501E0EE66E010ED5
:100D5000E66E57EC00F0E552E552F3CF16F7F4CF0C
:100D600017F72E0EE66E8EEC00F0E552040EDBCF88
:100D7000E6FF050EDBCFE6FF59EC02F0E552E55247
:100D8000060EE15C02E2E16AE552E16EE552E7CF70
:100D9000D9FF12000F01426B428F428B4289E80E4D
:100DA000E66E030EE66EE66AE66A72D8E552E55232
:100DB000E552E5520F01418F419D418B418741959D
:100DC00041954191406B1200D9CFE6FFE1CFD9FFA9
:100DD000E652800EDF6EDF50000813E2FE0EDB509D
:100DE000DF1406E0310EE66E8EEC00F0E55205D021
:100DF000300EE66E8EEC00F0E552DF407F0BDF6ECA
:100E0000EAD7E552E552E7CFD9FF1200D9CFE6FF86
:100E1000E1CFD9FF020EE126FE0EDB50F00BE838E1
:100E20000F0B300FDF6EDF50390803E2070EDF24AF
:100E3000DF6EFE0EDB500F0B300FE76E010EE7CFBB
:100E4000DBFFDB5039080AE2070E146E010EDBCF20
:100E5000E7FF1450E726010EE7CFDBFFDFCFE6FF09
:100E60008EEC00F0E552010EDBCFE6FF8EEC00F0D9
:100E7000E552680EE66E8EEC00F0E552020EE15C83
:100E800002E2E16AE552E16EE552E7CFD9FF1200D6
:100E9000D9CFE6FFE1CFD9FFFB0EDBCF05F0FC0E8B
:100EA000DBCF06F0FD0EDBCF07F0FE0EDBCF08F048
:100EB0000834000E081809E6D880000E0554000E0C
:100EC0000654000E0754000E08540CE2D950FB0FD4
:100ED000E96EFF0EDA20EA6EEE06000EEE5AEE5ACA
:100EE000EE5ADAD7E552E7CFD9FF1200D9CFE6FFA5
:100EF000E1CFD9FF020EE126DE6ADD6ADECF14F013
:100F0000DDCF15F0FE0EDB50000115AE02D0D890FB
:100F100003D0145C000E15580AE2200EE66E8EEC2B
:100F200000F0E552DF2A010E01E3DB2AE7D7020ECB
:100F3000E15C02E2E16AE552E16EE552E7CFD9FFFA
:100F40001200816893680F01396B070E806E386B51
:100F50003881388338850F0E926E806A82683A6BCA
:100F6000800E946E948E949C3B6B956A3C6B966855
:100F7000606A1200C280C19EC08EC08AC088C096BE
:100F8000C094C082C090C196C194C192C190120019
:100F9000D9CFE6FFE1CFD9FF040EE126FD0EDBCF6E
:100FA00014F0FE0EDBCF15F0D89014361536D8901D
:100FB00014361536010E1424C26E0A0EE66E2BECA2
:100FC0001BF0E55244EC1BF03FEC1BF0000901E084
:100FD000FBD736EC1BF0F3CFDEFFF4CFDDFF5EC1B5
:100FE000E6FF5FC1E6FFDECFE6FFDDCFE6FF94EC74
:100FF00015F0E552E552E552E5524D0EE66E8EECE7
:1010000000F0E552FD0EDBCF14F0FE0EDBCF15F045
:10101000300E1424E66E8EEC00F0E5523D0EE66EC6
:101020008EEC00F0E5525EC1E6FF5FC1E6FF57ECD3
:1010300000F0E552E552020EF3CFDBFF030EF4CFD2
:10104000DBFF880EE66E130EE66EE66AE66A20DFC8
:10105000E552E552E552E552DECF14F0DDCF15F052
:1010600014C0F3FF15C0F4FF040EE15C03E200D0EE
:10107000E16AE552E16EE552E7CFD9FF1200CD9E5D
:10108000CD9CCD8ACD88CD96CD94CD82CD90CC9E71
:10109000CC9ACC92CC909F80D08EDB0EE66E0B0E5D
:1010A000E66EC8EC1AF0E552E5529E90F29CCD90A7
:1010B0009D90F29EF29C1200D9CFE6FFE1CFD9FFBE
:1010C000020EE126DE6ADD6AFB0EDBCFF6FFDB2ACD
:1010D000FC0EDBCFF7FF01E3DB2A0800F550E66EDC
:1010E000FD0EDBCFE9FFDB2AFE0EDBCFEAFF01E3DB
:1010F000DB2AE552E750EF6EDF2A010E01E3DB2A1F
:10110000DECF14F0DDCF15F0D890155004E6000EB8
:10111000145C010E1558D8E3020EE15C02E2E16AAC
:10112000E552E16EE552E7CFD9FF1200D9CFE6FFD5
:10113000E1CFD9FF020EE126DE6ADD6AFB0EDBCFCE
:10114000F6FFDB2AFC0EDBCFF7FF01E3DB2A08000A
:10115000F550E66EFF0EE76EFD0EDBCF14F0FE0ECF
:10116000DBCF15F0E7501426000E1522DE50145C7C
:10117000E96EDD501558EA6EE552E750EF6EDF2A52
:10118000010E01E3DB2ADECF14F0DDCF15F0D8909D
:10119000155004E6000E145C010E1558CFE3020E44
:1011A000E15C02E2E16AE552E16EE552E7CFD9FF88
:1011B0001200980EE66E3A0EE66EE66AE66A68DEA1
:1011C000E552E552E552E552BCDE0701700E046FB0
:1011D000010E056F04C702F705C703F701011E0ED4
:1011E0005E6F010E5F6F07017C6B7D6B7E6B7F6BAB
:1011F000816B818D818981958197819181930F6B1D
:10120000106B0D6B0E6B886B896B0EEC00F00C0E87
:10121000E66E8EEC00F0E552A00EE66E860EE66EEF
:10122000010EE66EE66A34DEE552E552E552E5521D
:101230009EEC00F05EC1E6FF5FC1E6FF57EC00F0F8
:10124000E552E552F3CF16F7F4CF17F79EEC00F016
:1012500002C114F003C115F0166A14C0E6FF15C0F0
:10126000E6FF16C0E6FF1E0EE66E010EE66E49ECC6
:101270001AF0176E050EE15E17501E0EE66E010E97
:10128000E66E57EC00F0E552E552F3CF16F7F4CFD7
:1012900017F79EEC00F0100EE66E270EE66EE66A7B
:1012A000E66AF6DDE552E552E552E5521AC114F060
:1012B0001BC115F0166A14C0E6FF15C0E6FF16C084
:1012C000E6FF1E0EE66E010EE66E49EC1AF0176E92
:1012D000050EE15E17501E0EE66E010EE66E57EC2F
:1012E00000F0E552E552F3CF16F7F4CF17F79EEC76
:1012F00000F016C114F017C115F0166A14C0E6FF0D
:1013000015C0E6FF16C0E6FF1E0EE66E010EE66E85
:1013100049EC1AF0176E050EE15E17501E0EE66ED0
:10132000010EE66E57EC00F0E552E552F3CF16F7EA
:10133000F4CF17F718C114F019C115F0166A14C0CC
:10134000E6FF15C0E6FF16C0E6FF1E0EE66E010EB4
:10135000E66E49EC1AF0176E050EE15E17501E0E90
:10136000E66E010EE66E57EC00F0E552E552F3CF63
:1013700016F7F4CF17F7000EE66EE66A0DEC02F0F2
:10138000E552E5529EEC00F014C114F015C115F0C1
:10139000166A14C0E6FF15C0E6FF16C0E6FF1E0E73
:1013A000E66E010EE66E49EC1AF0176E050EE15E70
:1013B00017501E0EE66E010EE66E57EC00F0E55279
:1013C000E552F3CF16F7F4CF17F7880EF66E280E16
:1013D000F76E0900F5CF64F70900F5CF65F709004E
:1013E000F5CF66F70800F5CF67F7060EE66E5EC12B
:1013F000E6FF5FC1E6FF64C7E6FF65C7E6FF66C7B5
:10140000E6FF67C7E6FFB4EC02F0146E070EE15E7C
:1014100014505EC1E6FF5FC1E6FF57EC00F0E552F5
:10142000E552F3CF16F7F4CF17F79EEC00F0B2DCDD
:10143000A1DD0701866B876BE66A010EE66E880EFA
:10144000146E240E156E166A14C0E6FF15C0E6FF72
:1014500016C0E6FF000EE66E060EE66E26EC1AF0EB
:10146000176E070EE15E175012C114F013C115F08C
:10147000166A14C0E6FF15C0E6FF16C0E6FF1E0E92
:10148000E66E010EE66E49EC1AF0176E050EE15E8F
:1014900017501E0EE66E010EE66E57EC00F0E55298
:1014A000E552F3CF16F7F4CF17F707017C6B7D6B8E
:1014B0007E6B7F6B0101E80E9A6F030E9B6F9C6B36
:1014C0009D6B9AC104F09BC105F09CC106F09DC1C3
:1014D00007F058EC0FF005C060F706C061F707C0D1
:1014E00062F708C063F7880EF66E280EF76E0900E3
:1014F000F5CF64F70900F5CF65F70900F5CF66F77A
:101500000800F5CF67F764C70AF065C70BF066C738
:101510000CF067C70DF060C705F061C706F062C741
:1015200007F063C708F00AEC10F005C05CF706C0CE
:101530005DF707C05EF708C05FF75CC7E6FF5DC7F1
:10154000E6FF5EC7E6FF5FC7E6FF4FEC19F0E55226
:10155000E552E552E55204C014F005C015F006C08E
:1015600016F007C017F014C005F015C006F016C03D
:1015700007F017C008F020EC11F004C078F705C0A0
:1015800079F706C07AF707C07BF71E0EE66E010EEC
:10159000E66E78C7E6FF79C7E6FF7AC7E6FF7BC746
:1015A000E6FF2EEC16F0146E060EE15E14501E0ED1
:1015B000E66E010EE66E57EC00F0E552E552F3CF11
:1015C00016F7F4CF17F79EEC00F0100EE66E270E1C
:1015D000E66EE66AE66A5CDCE552E552E552E55203
:1015E000D08ED09CAB889D8AF28CF28EF28C070153
:1015F000846B856B116B07010451021902E10551DF
:10160000031901E1D0D2A7EC00F00701076F842B8A
:10161000000E85230751580A01E1D6D10A0A01E1DB
:1016200082D1160A01E12FD1100A01E18CD0170AEC
:101630005AE0100A01E0B7D2200EE66EE66A0DEC21
:1016400002F0E552E5520701126B136B000E125DBA
:10165000010E135946E2880E1225F66E240E132150
:10166000F76E0800F5CF18F018C007F032EC0FF055
:1016700005C014F006C015F007C016F008C017F03A
:101680000A6A0B6A0C6A410E0D6E14C005F015C093
:1016900006F016C007F017C008F00AEC10F005C0FD
:1016A0006CF706C06DF707C06EF708C06FF76CC720
:1016B00005F06DC706F06EC707F06FC708F0CAECFB
:1016C00010F00750E66E000E07011225E96E060EB7
:1016D0001321EA6EE552E750EF6E122B000E132332
:1016E000B5D7116B60D2400EE66EE66A0DEC02F0E3
:1016F000E552E5520701126B136B800E125D000E6E
:1017000013590CE2000E1225E96E060E1321EA6E43
:101710001F0EEF6E122B000E1323EFD7800E126FE9
:10172000136B000E125D010E13590BE2000E122511
:10173000E96E060E1321EA6EEF6A122B000E1323D8
:10174000F0D7116B30D2600EE66EE66A0DEC02F057
:10175000E552E5520701126B136B800E125D000E0D
:1017600013593FE212C706F013C707F043EC0FF01E
:1017700005C014F006C015F007C016F008C017F039
:101780000A6A0B6A0C6A410E0D6E14C005F015C092
:1017900006F016C007F017C008F00AEC10F005C0FC
:1017A0006CF706C06DF707C06EF708C06FF76CC71F
:1017B00005F06DC706F06EC707F06FC708F0CAECFA
:1017C00010F00750E66E000E07011225E96E060EB6
:1017D0001321EA6EE552E750EF6E122B000E132331
:1017E000BCD7800E126F136B000E125D010E1359E1
:1017F00048E212C718F013C719F0000ED880185627
:10180000010E195618C006F019C007F043EC0FF08E
:1018100005C014F006C015F007C016F008C017F098
:101820000A6A0B6A0C6A410E0D6E14C005F015C0F1
:1018300006F016C007F017C008F00AEC10F005C05B
:101840006CF706C06DF707C06EF708C06FF76CC77E
:1018500005F06DC706F06EC707F06FC708F0CAEC59
:1018600010F00750E66E000E07011225E96E060E15
:101870001321EA6EE552E750EF6E122B000E132390
:10188000B3D7116B90D1800EE66EE66A0DEC02F0D4
:10189000E552E5520701126B136B000E125D010E4B
:1018A00013593FE212C706F013C707F043EC0FF0DD
:1018B00005C014F006C015F007C016F008C017F0F8
:1018C0000A6A0B6A0C6A410E0D6E14C005F015C051
:1018D00006F016C007F017C008F00AEC10F005C0BB
:1018E0006CF706C06DF707C06EF708C06FF76CC7DE
:1018F00005F06DC706F06EC707F06FC708F0CAECB9
:1019000010F00750E66E000E07011225E96E060E74
:101910001321EA6EE552E750EF6E122B000E1323EF
:10192000BCD7116B40D1A00EE66EE66A0DEC02F05A
:10193000E552E55207011269136B000ED88012556B
:10194000000E13553FE212C706F013C707F043EC31
:101950000FF005C014F006C015F007C016F008C05F
:1019600017F00A6A0B6A0C6A410E0D6E14C005F07E
:1019700015C006F016C007F017C008F00AEC10F00A
:1019800005C06CF706C06DF707C06EF708C06FF7AB
:101990006CC705F06DC706F06EC707F06FC708F09B
:1019A000CAEC10F00750E66E000E07011225E96E32
:1019B000060E1321EA6EE552E750EF6E1207000E95
:1019C000135BBBD7116BEFD0C00EE66EE66A0DEC71
:1019D00002F0E552E552010EC26E0A0EE66E2BECE5
:1019E0001BF0E55244EC1BF03FEC1BF0000901E05A
:1019F000FBD736EC1BF0F3CF18F7F4CF19F718C765
:101A000006F019C707F043EC0FF005C018F006C048
:101A100019F007C01AF008C01BF00A6A0B6AC80E5A
:101A20000C6E420E0D6E18C005F019C006F01AC0FB
:101A300007F01BC008F05DEC10F005C014F006C004
:101A400015F007C016F008C017F00A6A0B6A800E7E
:101A50000C6E440E0D6E14C005F015C006F016C0D5
:101A600007F017C008F00AEC10F005C068F706C0D0
:101A700069F707C06AF708C06BF70701D8901933F8
:101A80001833D89019331833000ED8801855000E2B
:101A9000195501E384D0FF0E185D000E195901E3BA
:101AA0007ED0126B136B1851125D195113590CE251
:101AB000000E1225E96E060E1321EA6E1F0EEF6E60
:101AC000122B000E1323EFD718C712F719C713F7FD
:101AD000000E125D010E13590BE2000E1225E96E85
:101AE000060E1321EA6EEF6A122B000E1323F0D7B5
:101AF0005EC1E6FF5FC1E6FF18C7E6FF19C7E6FF54
:101B000094EC15F0E552E552E552E5524D0EE66EC5
:101B10008EEC00F0E552300E07011425E66E8EECD7
:101B200000F0E5523D0EE66E8EEC00F0E5525EC12F
:101B3000E6FF5FC1E6FF57EC00F0E552E552F3CF58
:101B400016F7F4CF17F7090EE66E8EEC00F0E552AB
:101B5000020EE66E5EC1E6FF5FC1E6FF68C7E6FF04
:101B600069C7E6FF6AC7E6FF6BC7E6FFB4EC02F0A1
:101B7000146E070EE15E14505EC1E6FF5FC1E6FF22
:101B800057EC00F0E552E552F3CF16F7F4CF17F714
:101B9000250EE66E8EEC00F0E5520701116B03D0C6
:101BA0000701846B856B050ED8808455000E855522
:101BB00001E3FDD00D0E075D01E0F9D0866B876B68
:101BC000126B136B050E125D000E135918E2700EA6
:101BD0001225E96E010E1321EA6EEF50E66EE66AF9
:101BE000FBEC1AF0E552E55207018651F324866FAB
:101BF0008751F420876F122B000E1323E3D7050EB5
:101C0000861901E187512EE010C114F011C115F0C1
:101C1000166A14C0E6FF15C0E6FF16C0E6FF1E0EEA
:101C2000E66E010EE66E49EC1AF0176E050EE15EE7
:101C300017501E0EE66E010EE66E57EC00F0E552F0
:101C4000E552F3CF16F7F4CF17F7C40EE66E090E80
:101C5000E66EE66AE66A48EC07F0E552E552E552C0
:101C6000E55299D0786B796B7A6B7B6B0101756B60
:101C7000700EE66E010EE66EE9EC14F0E552E552E8
:101C800004C09AF105C09BF106C09CF107C09DF10C
:101C90009AC104F09BC105F09CC106F09DC107F0FC
:101CA00058EC0FF005C060F706C061F707C062F797
:101CB00008C063F7880EF66E280EF76E0900F5CFA0
:101CC00064F70900F5CF65F70900F5CF66F708005E
:101CD000F5CF67F764C70AF065C70BF066C70CF06D
:101CE00067C70DF060C705F061C706F062C707F06F
:101CF00063C708F00AEC10F005C05CF706C05DF79A
:101D000007C05EF708C05FF75CC705F05DC706F067
:101D10005EC707F05FC708F020EC11F004C078F749
:101D200005C079F706C07AF707C07BF7010EE66EAB
:101D30005EC1E6FF5FC1E6FF60C7E6FF61C7E6FF81
:101D400062C7E6FF63C7E6FFB4EC02F0146E070E4D
:101D5000E15E14505EC1E6FF5FC1E6FF57EC00F0A4
:101D6000E552E552F3CF16F7F4CF17F7480EE66EBB
:101D70008EEC00F0E5527A0EE66E8EEC00F0E55245
:101D800078C78DF779C78CF77AC78BF707017C6B1B
:101D90007D6B7E6B7F6B0701700E046F010E056F0C
:101DA00004C702F705C703F7846B856B116B103509
:101DB00004E20F510008000E105507E30E3504E24F
:101DC0000D510008000E0E5521E200C1E6FF01C1D1
:101DD000E6FF1EEC00F0E552E552F3CF0BF7F4CF2F
:101DE0000CF70FC7E6FF10C7E6FF59EC02F0E5520B
:101DF000E552090EE66E8EEC00F0E5520DC7E6FFE7
:101E00000EC7E6FF59EC02F0E552E5520701146BEC
:101E1000156B7E51EA6A000FE96E060EEA22EFCFDB
:101E200040FF780EE96E070EEA6E7C51EE247C6F5F
:101E30007D51EE207D6F7E51EE207E6F7F51EE2032
:101E40007F6F1151E6E0C40EE66E090EE66EE66A9B
:101E5000E66A48EC07F0E552E552E552E552FBEF41
:101E60000AF012000F9E05D00F9E07AE02D0076C3D
:101E70000F8E07C001F0006A136A126A860E026EA6
:101E8000036ADAEF11F00F9E08D00F9E07AE05D05F
:101E9000066C071EE86A07220F8E07C001F006C015
:101EA00000F0136A126A8E0E026E036ADAEF11F006
:101EB0000F9E0CD00F9E07AE09D0046C051E061EA7
:101EC000071EE86A0522062207220F8E07C001F0CE
:101ED00006C000F005C013F004C012F09E0E026EA2
:101EE000036ADAEF11F00D7E0F6A16EC12F02EEC99
:101EF00012F00FB6BEEF11F00FA20AD00FAA03D056
:101F00000FBEBEEF11F00FA4CAEF11F0C7EF11F032
:101F10000FAA05D00FACCAEF11F0C7EF11F00FA058
:101F20000AD00FA808D00FBE04D00FA402D0D3EF60
:101F300011F0D7EF11F0126A036A0D50085C116EB0
:101F400010E305C013F006C000F007C001F008C0A0
:101F500010F00AC005F00BC006F00CC007F00F3AF5
:101F600009D00AC013F00BC000F00CC001F00DC086
:101F700010F0116C0F9E0FBC0F8E10C002F00FB04E
:101F800006EF12F01A0E116006EF12F0026A086AEC
:101F90000FA408D0056C061E071E081EE86A06225C
:101FA000072208220FAC08D0136C001E011E021E6F
:101FB000E86A002201220222046A115207E0083472
:101FC0000732063205320432112EF9D70550132696
:101FD00006500022075001220850022204C012F0CD
:101FE0000F9E02AE0BD0126C131E001E011E021EAD
:101FF000E86A13220022012202220F8E02A006D0DC
:10200000D8800132003213321232102A10C002F08E
:10201000DAEF11F00F6A16EC12F02EEC12F00FB698
:10202000BEEF11F00FA205D00FBABEEF11F0C5EF51
:1020300011F00FBAD1EF11F00FA005D00FB8BEEF1D
:1020400011F0D1EF11F00FB8C5EF11F0036A7F0E58
:102050000824026EE86A03220D50025EE86A035A01
:102060001A0E106E086A126A136A006A016A0A5030
:10207000055E0B50065A0C50075A000E085A09E725
:102080000A5005260B5006220C500722000E08228B
:1020900001D0128AD8900536063607360836D89011
:1020A0001236133600360136102EE1D707500610CF
:1020B0000510D8A4128ADAEF11F00F6A16EC12F0AC
:1020C0002EEC12F00FB6BEEF11F00FA205D00FB834
:1020D000BEEF11F0C5EF11F00FAA05D00FB0BEEFA3
:1020E00011F0C5EF11F00FB002D00FA802D0D1EF60
:1020F00011F0036A0D500824026EE86A03227E0E76
:10210000025EE86A035A126A136A006A016A0C5096
:102110000702F4CF01F0F3CF00F00B500702F350A9
:102120001326F4500022000E01220C500602F35038
:102130001326F4500022000E01220A500702F35029
:102140001226F4501322000E002201220B50060228
:10215000F3501226F4501322000E002201220C50DC
:102160000502F3501226F4501322000E0022012221
:102170000A500602F4501226000E132200220122F9
:102180000B500502F4501226000E132200220122E9
:10219000DAEF11F00F6A16EC12F00FB6D4EF10F070
:1021A0000FA20AD00FB403D07F0E076E19D0800E95
:1021B000076E16D0076A14D00FB0FCD7870E0860E0
:1021C000F1D77E0E0864F6D7860E085C04E0D8903E
:1021D0000732082AF9D70FA403D0076C07AEEAD755
:1021E00012000F6A16EC12F00FB6FBEF10F00FA200
:1021F0000ED00FB405D07F0E076EFF0E066E1FD0F7
:10220000800E076E066A1BD0076A066A18D00FB0E8
:10221000FBD78F0E0860EDD77E0E0864F5D78E0EC3
:10222000085C05E0D89007320632082AF8D70FA4D8
:1022300006D0066C071EE86A072207AEE5D7120033
:102240000F6A16EC12F00FB62AEF11F00FA20FD0A2
:102250000FB407D07F0E076EFF0E066E056E046E7C
:1022600025D0800E076E01D0076A000EF6D70FB09A
:10227000FBD7046A9F0E0860EBD77E0E0864F4D784
:102280009E0E085C07E0D890073206320532043211
:10229000082AF6D70FA40AD0046C051E061E071ED6
:1022A000E86A05220622072207AEDED7120069EC93
:1022B00011F00FB6000C0FB0000C0FB4000C010CA5
:1022C00069EC11F00FB6000C0FB0000C0FA4000C5D
:1022D000010C0F6A16EC12F02EEC12F00FB6120081
:1022E0000FAE08D00FA004D00FA802D00F801200AC
:1022F0000F9012000D50085C0BE10C50075C08E1D8
:102300000B50065C05E10A50055C02E10F801200EB
:10231000D8A002D00F8E10D008500DC008F00D6E5E
:1023200007500CC007F00C6E06500BC006F00B6E89
:1023300005500AC005F00A6E0D50085C10E0FF0F52
:1023400009E00F900FB403D00FAE0F8412000FAE50
:102350000F9412000D2AD8900C320B320A320A5018
:10236000055E0B50065A0C50075A07BEEAD7D890A4
:10237000053606360736082EF8D7C8D77F0E086E02
:10238000FF0E076E066E056E12007F0E0FBEFF0E6B
:10239000086E02D07F0E086E800E076E066A056A10
:1023A000F3D70FAE04D0800E086E076AF7D7086A1D
:1023B000076AF4D70150001013101210F8E003BEA2
:1023C000F0D701BE0CD002500310EBE0D8901236CB
:1023D0001336003601360206D8A00306F2D70350A2
:1023E000D4E10228D2E012AE11D07F0E121402E125
:1023F00013A00CD0132AE86A0022012207E3D88038
:10240000013200321332022A0228BFE00250C9E032
:1024100013C005F000C006F00134076E0230086EEC
:102420000732089E0FBE088EC4EF11F0073608363B
:1024300002E30F840F7E06E10F80086A076A066ACE
:10244000056A1200082803E0D88007321200D890ED
:10245000073202E10F8212000F8612000C360D3691
:1024600002E30F8C0F7E06E10F880D6A0C6A0B6A7F
:102470000A6A12000D2803E0D8800C321200D890AE
:102480000C32EAE10F8A1200808285888B8E91944B
:10249000979A9DA0A2A5A8ABADB0B3B5B8BBBDC07F
:1024A000C2C5C7C9CCCED0D2D4D6D8DADCDEE0E201
:1024B000E3E5E6E8E9EBECEDEEEFF0F1F2F3F4F54D
:1024C000F5F6F6F7F7F7F7F7F8F7F7F7F7F7F6F6A1
:1024D000F5F5F4F3F2F1F0EFEEEDECEBE9E8E6E51B
:1024E000E3E2E0DEDCDAD8D6D4D2D0CECCC9C7C5A0
:1024F000C2C0BDBBB8B5B3B0ADABA8A5A2A09D9AF4
:102500009794918E8B888582807D7A7774716E6BBB
:102510006865625F5D5A5754524F4C4A4744423F88
:102520003D3A383633312F2D2B29272523211F1DE6
:102530001C1A19171614131211100F0E0D0C0B0A7A
:102540000A09090808080808080808080808090905
:102550000A0A0B0C0D0E0F10111213141617191A6C
:102560001C1D1F21232527292B2D2F313336383AC7
:102570003D3F4244474A4C4F5254575A5D5F626553
:10258000686B6E7174777A7D00010203040506079B
:1025900008090A0B0C0D0E0F101112131415161743
:1025A00018191A1B1C1D1E1F202122232425262733
:1025B00028292A2B2C2D2E2F303132333435363723
:1025C00038393A3B3C3D3E3F404142434445464713
:1025D00048494A4B4C4D4E4F505152535455565703
:1025E00058595A5B5C5D5E5F6061626364656667F3
:1025F00068696A6B6C6D6E6F7071727374757677E3
:1026000078797A7B7C7D7E7F8081828384858687D2
:1026100088898A8B8C8D8E8F9091929394959697C2
:1026200098999A9B9C9D9E9FA0A1A2A3A4A5A6A7B2
:10263000A8A9AAABACADAEAFB0B1B2B3B4B5B6B7A2
:10264000B8B9BABBBCBDBEBFC0C1C2C3C4C5C6C792
:10265000C8C9CACBCCCDCECFD0D1D2D3D4D5D6D782
:10266000D8D9DADBDCDDDEDFE0E1E2E3E4E5E6E772
:10267000E8E9EAEBECEDEEEFF0F1F2F3F4F5F6F762
:10268000F8F9FAFBFCFDFEFFFFFFFFFFFFFFFFFF76
:10269000FFFFFFFFFFFFFFFFFFFFFFFFFFFFFFFF4A
:1026A000FFFFFFFFFFFFFFFFFFFFFFFFFFFFFFFF3A
:1026B000FFFFFFFFFFFFFFFFFFFFFFFFFFFFFFFF2A
:1026C000FFFFFFFFFFFFFFFFFFFFFFFFFFFFFFFF1A
:1026D000FFFFFFFFFFFFFFFFFFFFFFFFFFFFFFFF0A
:1026E000FFFFFFFFFFFFFFFFFFFFFFFFFFFFFFFFFA
:1026F000FFFFFFFFFFFFFFFFFFFFFFFFFFFFFFFFEA
:10270000FFFFFFFFFFFFFFFF0000000000000000D1
:1027100000000000000000000000000000000000B9
:1027200000000000000000000000000000000000A9
:102730000000000000000000000000000000000099
:102740000000000000000000000000000000000089
:102750000000000000000000000000000000000079
:102760000000000000000000000000000000000069
:102770000000000000000000000000000000000059
:10278000000000000000000008090B0D0F111315D8
:1027900017181A1C1E2022242627292B2D2F3133EF
:1027A0003536383A3C3E4042444547494B4D4F51FF
:1027B000535456585A5C5E6062636567696B6D6F0F
:1027C00071727476787A7C7E8081838587898B8D1F
:1027D0008F90929496989A9C9E9FA1A3A5A7A9AB2F
:1027E000ADAEB0B2B4B6B8BABCBDBFC1C3C5C7C93F
:1027F000CBCCCED0D2D4D6D8DADBDDDFE1E3E5E74F
:10280000E9EAECEEF0F2F4F6F8F6F4F2F0EEECEAC7
:10281000E9E7E5E3E1DFDDDBDAD8D6D4D2D0CECC10
:10282000CBC9C7C5C3C1BFBDBCBAB8B6B4B2B0AEE0
:10283000ADABA9A7A5A3A19F9E9C9A9896949290B0
:102840008F8D8B8987858381807E7C7A7876747280
:10285000716F6D6B6967656362605E5C5A58565450
:1028600053514F4D4B4947454442403E3C3A383620
:102870003533312F2D2B2927262422201E1C1A18F0
:10288000171513110F0D0B094CD8B43C4672616D2E
:102890006520457272657572206574204F76657289
:1028A000666C6F7720646574656374696F6E203A37
:1028B0002000506F727420636F6D6D203338343098
:1028C00030626473206F7576657274004D61727149
:1028D000756572203225206475207369676E616C9E
:1028E0000045534320706F757220736F7274697264
:1028F0000D004361707475726520546175782073A2
:10290000757220414443302000536F727469652012
:102910004E6F726D616C6520646520507267006354
:1029200061722072656375203A0055736167652096
:10293000513D31304D687A2078342028504C4C2954
:102940000D00457272657572205361697369652E59
:102950002E2E2E2E0D00496E697420436F6E734625
:1029600072657120314B687A090046616374657540
:102970007220444453203D2000436F6E7369676E9C
:10298000652076696120436C61766965720D005639
:10299000657273696F6E20312E2E343030303048BE
:1029A0007A200D004331383A31384634364B3232D2
:1029B0005F4444535F5354435844524D5F31323067
:1029C0003730355F41444335625F4331382E630D04
:1029D00000FFFF0EE3CFEAFFE552FF0EE3CFE9FF72
:1029E000E552E66AE66AE66AE66AD9CFE6FFDACF3A
:1029F000E6FFFA0EE124D96EFF0EE220DA6EE66AF7
:102A0000E66AE66AE66AE66A200EEF5C06E0090E10
:102A1000EF5C03E0EF6603D06BD0EE50F5D72D0EE0
:102A2000EF5C03E1FF0EE32A03D02B0EEF5C01E124
:102A3000EE502F0EEF6444D03A0EEF6041D0D890A4
:102A4000F50EE336F60EE336F70EE336F80EE33610
:102A5000FB0EDECFE3FFFC0EDECFE3FFFD0EDECF8D
:102A6000E3FFFE0EDDCFE3FFDD52DD52D890F50E21
:102A7000E336F60EE336F70EE336F80EE336D8907B
:102A8000F50EE336F60EE336F70EE336F80EE336D0
:102A9000FB0EE350DE26FC0EE350DE22FD0EE3507B
:102AA000DE22FE0EE350DD22DD52DD52300EEE5C02
:102AB000DE26000EDE22DE22DD22DD52DD52B9D717
:102AC000FF0EE3CFE8FFE85213E0F50EE31EF60E2B
:102AD000E31EF70EE31EF80EE31EF50EE32A08E1EF
:102AE000F60EE32A05E1F70EE32A02E1F80EE32AE7
:102AF000E552E552E552E552E552D9CFE9FFDACF8A
:102B0000EAFFEECF04F0EECF05F0EECF06F0EFCF08
:102B100007F0FF0EE3CFDAFFE552FF0EE3CFD9FF58
:102B2000E552E552E5521200D9CFE6FFDACFE6FFD3
:102B3000FA0EE3CFD9FFFB0EE3CFDAFFFD0EE3522F
:102B400009E72D0EDE6EFC0EE31EE32AFD0ED8B45F
:102B5000E306E31EE652E652E652FD0EE124E76E7E
:102B6000FF0EE220E46EE652F70EE3CFE6FFF70E2B
:102B7000E3CFE6FF04EC16F0F90EE124E96EFF0E58
:102B8000E220EA6EF4EC15F00AE1F1EC15F009E14F
:102B9000F4EC15F008E1F1EC15F007E108D0FFECDA
:102BA00015F0FAEC15F0FFEC15F0FAEC15F0FFEC6F
:102BB00015F0DE6AF90EE126FF0EE222FF0EE3CFEA
:102BC000DAFFE552FF0EE3CFD9FFE552FC0EE12418
:102BD000E96EFF0EE220EA6EEECFF3FFEFCFF4FFD7
:102BE0001200EF380F0B1200EF500F0B02E1EE5204
:102BF000D8841200EF380F0B300FDE6E1200EE504B
:102C00000F0B300FDE6E1200FC0EE3CFE9FFFD0E5E
:102C1000E3CFEAFF100EE66EEE6AEE6AEF6AD89036
:102C2000FD0EE336FE0EE336ED36ED36EF36FF0EE3
:102C3000E30609E025EC16F0EE5225EC16F0EE5214
:102C400025EC16F0EDD7E56E1200030EEF24E8B682
:102C5000EF6E300EEF24E8BEEF6E000CD9CFE6FF2A
:102C6000DACFE6FFF80EE3CFD9FFF90EE3CFDAFFB4
:102C7000E652E652E652E652E652FB0EE124E76ED9
:102C8000FF0EE220E46EE652F30EE3CFE6FFF30E12
:102C9000E3CFE6FFF30EE3CFE6FFF30EE3CFE6FF6D
:102CA000B3EC16F0F50EE124E96EFF0EE220EA6EB9
:102CB000A0EC16F019E1A3EC16F018E1A0EC16F068
:102CC00017E1A3EC16F016E1A0EC16F015E1A3EC69
:102CD00016F014E1A0EC16F013E1A3EC16F012E1EB
:102CE000A0EC16F011E112D0A9EC16F0AEEC16F043
:102CF000A9EC16F0AEEC16F0A9EC16F0AEEC16F05E
:102D0000A9EC16F0AEEC16F0A9EC16F0AEEC16F04D
:102D1000DE6AF50EE126FF0EE222FF0EE3CFDAFFB8
:102D2000E552FF0EE3CFD9FFE552FA0EE124E96E3A
:102D3000FF0EE220EA6EEECFF3FFEFCFF4FF1200BA
:102D4000EF380F0B1200EF500F0B02E1EE52D88458
:102D50001200EF380F0B300FDE6E1200EE500F0B2B
:102D6000300FDE6E1200FA0EE3CFE9FFFB0EE3CF69
:102D7000EAFF200EE66EEE6AEE6AEE6AEE6AEF6A2F
:102D8000D890FB0EE336FC0EE336FD0EE336FE0E66
:102D9000E336ED36ED36ED36ED36EF36FF0EE30673
:102DA0000FE0E2EC16F0EE52E2EC16F0EE52E2EC3E
:102DB00016F0EE52E2EC16F0EE52E2EC16F0E1D72D
:102DC000E56E1200030EEF24E8B6EF6E300EEF242E
:102DD000E8BEEF6E000CD9CFE6FFDACFE6FFE1CF19
:102DE000D9FFE2CFDAFF130EE12402E3E168E652F5
:102DF000E16E0C0EDB6AD950FA0FE96EFF0EDA2095
:102E0000EA6E080EEECFDBFF090EEECFDBFF0A0EF7
:102E1000EECFDBFF0B0EEECFDBFF1FD9D950080F33
:102E200017D9EECFE6FFEECFE6FFEECFE6FFEFCF0E
:102E3000E6FF34EC18F0146E060EE15C02E2E16A83
:102E4000E552E16E1450DF6E020EDF5C01E0BCD093
:102E5000050EDBCF16F0060EDBCF17F0F80EDB50B9
:102E6000165C146EF90EDB501758156E7F0E145E4B
:102E7000000E155A0D0E14C0DBFF0E0E15C0DBFF41
:102E80000D0E0E0EDBCF15F00001800E15140AE0BA
:102E9000010EF36E0C0EF3CFDBFF070EDB5001E0EB
:102EA00098D09DD00D0EDBCF14F00E0EDBCF15F0B9
:102EB000D890155004E6170E145C000E155801E367
:102EC0009ED0186819687F0E1A6E1B6A0D0EDB50B3
:102ED0001F0B18C014F019C015F01AC016F01BC053
:102EE00017F007E0D8901732163215321432E80680
:102EF000F9E10F0E14C0DBFF100E15C0DBFF110E41
:102F000016C0DBFF120E17C0DBFF0F0EDBCF14F075
:102F1000100EDBCF15F0110EDBCF16F0120EDBCF4B
:102F200017F0D950010F94D8EE501416EE50151624
:102F3000EE501616EE5017161450151016101710E6
:102F400002E1000E01D0010EE76E0C0EE7CFDBFFB1
:102F5000DB5055E0186A196A800E1A6E1B6A010E62
:102F60001C6E1D6A1E6A1F6AD9500F0F71D8EE5071
:102F70001C26EE501D22EE501E22EE501F221C5029
:102F8000185C146E1D501958156E1E501A58166E86
:102F90001F501B58176ED950010F5AD81450EE16F7
:102FA0001550EE161650EE161750EE16D950080FA3
:102FB000E66E000EDA20E66E50D8C2EC18F0E5524C
:102FC000E552E552E5521BD0DF0419E1070EDB5054
:102FD00006E0146A156A166A800E176E04D0146A29
:102FE000156A166A176A080E14C0DBFF090E15C0B1
:102FF000DBFF0A0E16C0DBFF0B0E17C0DBFFF60E61
:10300000DBCFE9FFF70EDBCFEAFF0C0EDBCFEFFFE4
:10301000080EDBCF14F0090EDBCF15F00A0EDBCF64
:1030200016F00B0EDBCF17F014C004F015C005F03E
:1030300016C006F017C007F0130EE15C02E2E16A69
:10304000E552E16EE552E5CFDAFFE7CFD9FF120096
:10305000E96E000EDA20EA6E1200D950010FE66E1A
:10306000000EDA20E66E1200D9CFE6FFDACFE6FFD7
:10307000E1CFD9FFE2CFDAFFE652146815687F0E80
:10308000166E176AD950FA0FE96EFF0EDA20EA6E53
:10309000EE501416EE501516EE501616EE5017168A
:1030A0006AD814C0EEFF15C0EEFF16C0EEFF17C0C1
:1030B000EEFFFD0EDB50800B02E0010E01D0000E92
:1030C000E66E59D8060EE926000EEA22E552E750D0
:1030D000EF6EFC0EDBCF14F0FD0EDBCF15F0D890B9
:1030E00014361536FC0E14C0DBFFFD0E15C0DBFFD9
:1030F000DB50E66E40D8040EE926000EEA22E552C7
:10310000E750EE6EED6AFD0EDB50146E156AFF0E91
:10311000141818E1155016E12ED8EECF14F0EECFAA
:1031200015F0EECF16F0EFCF17F014501510161063
:10313000171006E0210E0F010A6F0B6B800E0BD0EB
:10314000040E09D0FD0EDB5008E115D8EE6AEE6AD8
:10315000EE6AEE6A010EDF6E06D0020EDF6E0BD84D
:10316000EE52EE52EE8EDF50E552E552E5CFDAFF39
:10317000E7CFD9FF1200F80EDBCFE9FFF90EDBCF66
:10318000EAFF1200D9CFE6FFDACFE6FFE1CFD9FFA1
:10319000E2CFDAFF5BD8153411E21450FE08000EBE
:1031A00015540CE276D805E06CD8800EEE6EEE6811
:1031B00047D067D8800EEE6E7F0E0ED047D8D890DD
:1031C000155004E6010E145C000E15580BE261D890
:1031D00005E057D8EE6A800EEE6E32D052D8EE6A15
:1031E000EE6A2ED047D8EECF14F0EECF15F0EECF2A
:1031F00016F0EFCF17F032D814C0EEFF15C0EEFF77
:1032000016C0EEFF17C0EEFF21D81450010B05E0E9
:1032100025D8020E3AD8EF8E04D020D8020E35D829
:10322000EF9E14D8D8901532143218D8030E2DD82A
:1032300014C0EFFF1AD804E011D8030E26D8EF8E81
:10324000E552E5CFDAFFE7CFD9FF120013D8040E1D
:103250001CD8EECF14F0EFCF15F01200FA0EDBCF32
:10326000E9FFFB0EDBCFEAFF120004D8060E0DD8F3
:10327000EF501200FC0EDBCFE9FFFD0EDBCFEAFFC3
:103280001200ECDFEE6AEE6A1200E926000EEA2276
:103290001200220E0F010A6F0B6B35EF19F0D9CF18
:1032A000E6FFDACFE6FFE1CFD9FFE2CFDAFF060E85
:1032B000E12402E3E168E652E16ED950050FE66EC3
:1032C000000EDA20E66E000EE66EE66AD950FA0FBE
:1032D000E96EFF0EDA20EA6EEECFE6FFEECFE6FFF4
:1032E000EECFE6FFEFCFE6FFEBEC16F0146E080E24
:1032F000E15C02E2E16AE552E16E1450010E04C0A5
:10330000DBFF020E05C0DBFF030E06C0DBFF040E71
:1033100007C0DBFF050EDB502AE0040EDB50800BFC
:1033200026E1146A156A800E166E3F0E176ED9508C
:10333000010FE96E000EDA20EA6EEECF05F0EECF57
:1033400006F0EECF07F0EFCF08F014C00AF015C07A
:103350000BF016C00CF017C00DF074EC0FF008C0A5
:10336000EDFF07C0EDFF06C0EDFF05C0EFFF010E4A
:10337000DBCF14F0020EDBCF15F0030EDBCF16F01F
:10338000040EDBCF17F014C004F015C005F016C012
:1033900006F017C007F0060EE15C02E2E16AE552B2
:1033A000E16EE552E5CFDAFFE7CFD9FF12000E0E4E
:1033B000F66E000EF76E000EF86E0F010900F55064
:1033C000056F0900F550066F03E1056701D03DD098
:1033D0000900F550006F0900F550016F0900F55024
:1033E000026F09000900F550E96E0900F550EA6E18
:1033F000090009000900F550036F0900F550046F3A
:1034000009000900F6CF07FFF7CF08FFF8CF09FF43
:1034100000CFF6FF01CFF7FF02CFF8FF0F010353F4
:1034200002E1045307E00900F550EE6E0307F8E2ED
:103430000407F9D707CFF6FF08CFF7FF09CFF8FF4A
:103440000F010507000E065BBFD71200FB0EE3CF8E
:10345000F6FFFC0EE3CFF7FFFD0EE3CFF8FFFE0E05
:10346000E3CFE9FFFF0EE3CFEAFFE9CFF3FFEACFB7
:10347000F4FFF90EE35003E1FA0EE35009E0F90E10
:10348000E30602E2FA0EE3060900F5CFEEFFF1D7FC
:103490001200FB0EE3CFF6FFFC0EE3CFF7FFFD0EAD
:1034A000E3CFF8FFFE0EE3CFE9FFFF0EE3CFEAFF25
:1034B000E9CFF3FFEACFF4FF0900F5CFEFFFEE66A7
:1034C000FBD71200FE0EE3CFE9FFFF0EE3CFEAFFCA
:1034D000F36AF46AEE5203E0F34AF42AFBD71200CF
:1034E000D9CFE6FFDACFE6FFE1CFD9FFE2CFDAFFAF
:1034F000AC6AAB6AFD0EDBB0AC88DBA202D0AC8C50
:10350000AB8CDBB4AC8EDBA602D0AB8801D0AB8A2F
:10351000DBB8AC84DBBAAB86DBAC02D09D8A01D0D1
:103520009D9ADBAE02D09D8801D09D98FB0EDB50AA
:10353000AF6EFC0EDBCF15F015C014F0156A1450F9
:10354000B06EAC8AAB8EE552E5CFDAFFE7CFD9FF9C
:103550001200D9CFE6FFDACFE6FFE1CFD9FFE2CF05
:10356000DAFFE652F20E0F010C17ABAC03D00C9150
:10357000ABB00C81ABB40C85ABB20C87AE50DF6E38
:10358000DF50E552E552E5CFDAFFE7CFD9FF120071
:10359000D9CFE6FFDACFE6FFE1CFD9FFE2CFDAFFFE
:1035A000E652E652FC0EDBCFDEFFDBCFDDFF010E85
:1035B000DB50CF6EDF50CE6EE552E552E552E5CFDF
:1035C000DAFFE7CFD9FF1200D9CFE6FFDACFE6FF67
:1035D000E1CFD9FFE2CFDAFFACAC04D0AC900F0161
:1035E0000CB3AC80FD0EDB50AD6EE552E5CFDAFFDB
:1035F000E7CFD9FF1200F36AF46AFF0EE124E96E07
:10360000FF0EE220EA6EED6607D02F0EEF6404D0C5
:103610003A0EEF6001D0F32A1200380EF36E00EE7E
:1036200000F00F0E01D81200EA6002D0EE6AFCD75B
:10363000F350E9601200EE6AFCD71EEE00F02EEEA9
:1036400000F0F86A0F9CD7EC19F003EC00F0D9EC0D
:1036500008F0FBD71200FF0EE350E84E1200000006
:1036600000D000D000D0E82EFAD71200C450176E58
:10367000166AC3501610F36E17C0F4FF1200C25042
:10368000020B01E0010E1200C28212008C28B22847
:10369000CC28E128F22809291F292A29422956295C
:1036A0006A2979298F29A429882450524F4A4554E0
:1036B0003A2031384634364B32325F4444532E6D13
:1036C0006370200D000000000000000000000000FA
:1036D00000000000000000000000000000000000EA
:1036E000000000000000000000001E0131323334F1
:1036F00035363738393031323334350031323334BE
:103700003536373839303132333435360000000041
:1037100000000000000000000000000000000000A9
:103720000000000000000000000000000000FFFF9B
:10373000FFFFFFFFFFFFFFFFFFFFFFFFFFFFFFFF99
:10374000FFFFFFFFFFFFFFFFFFFFFFFFFFFFFFFF89
:10375000FFFFFFFFFFFFFFFFFFFFFFFFFFFFFFFF79
:10376000FFFFFFFFFFFFFFFFFFFFFFFFFFFFFFFF69
:0200000400F00A
:100000002031384634364B32322034304D687A2035
:1000100031304D487A7834202020504C4C0D00006F
:100020002053696E7573202020202020202020205E
:100030002020202020202020202020202000000020
:100040002043617272652020202020202020202063
:100050002020202020202020202020202000000000
:1000600020547269616E676C65202020202020205A
:1000700020202020202020202020202020000000E0
:100080002044656E742064652073636965202020B8
:1000900020202020202020202020202020000000C0
:1000A00020526576657273652064656E74206465A0
:1000B000207363696520202020202020200000007C
:1000C00020416363657320546175782076696120EF
:1000D000506F74617220202020202020200000001A
:1000E00020566F69653020706F757220312F323560
:1000F00036202061203235352F32353620200D0054
:10010000204D61727175657572202B2D34387074B5
:1001100073202F34382020202020202020000000B1
:10012000204D504C4142204944452056382E38330A
:100130002C4331382056332E34302E2020200D0011
:10014000FFFFFFFFFFFFFFFFFFFFFFFFFFFFFFFFBF
:10015000FFFFFFFFFFFFFFFFFFFFFFFFFFFFFFFFAF
:10016000FFFFFFFFFFFFFFFFFFFFFFFFFFFFFFFF9F
:10017000FFFFFFFFFFFFFFFFFFFFFFFFFFFFFFFF8F
:020000040030CA
:0E0000000032183C009984000FC00FE00F4042
:020000040020DA
:08000000FFFFFFFFFFFFFFFF00
:00000001FF
